BL51 BANKED LINKER/LOCATER V6.22.2.0                                                    03/13/2023  13:47:56  PAGE 1


BL51 BANKED LINKER/LOCATER V6.22.2.0, INVOKED BY:
C:\KEIL_V5\C51\BIN\BL51.EXE .\Release\system_FE81001.obj, .\Release\STARTUP.obj, .\Release\main.obj TO .\Release\Sample_
>> DrvSPI_Master REGFILE (.\Release\Sample_DrvSPI_Master.ORC) PRINT (.\Sample_DrvSPI_Master.m51) RAMSIZE (256) CODE (0X0
>> 000-0X1FFF) XDATA (0X8000-0X87FF)


MEMORY MODEL: SMALL


INPUT MODULES INCLUDED:
  .\Release\system_FE81001.obj (SYSTEM_FE81001)
  .\Release\STARTUP.obj (?C_STARTUP)
  .\Release\main.obj (MAIN)
  C:\KEIL_V5\C51\LIB\C51S.LIB (?C_INIT)
  C:\KEIL_V5\C51\LIB\C51S.LIB (?C_IBP)


LINK MAP OF MODULE:  .\Release\Sample_DrvSPI_Master (SYSTEM_FE81001)


            TYPE    BASE      LENGTH    RELOCATION   SEGMENT NAME
            -----------------------------------------------------

            * * * * * * *   D A T A   M E M O R Y   * * * * * * *
            REG     0000H     0008H     ABSOLUTE     "REG BANK 0"
            DATA    0008H     0004H     UNIT         ?DT?MAIN
            DATA    000CH     0002H     UNIT         ?DT?DELAY?MAIN
            DATA    000EH     0002H     UNIT         ?DT?_SPI_READBYTE?MAIN
            DATA    0010H     0001H     UNIT         ?DT?_SPI_WRITEBYTE?MAIN
            DATA    0011H     0001H     UNIT         ?C?LIB_DATA
            IDATA   0012H     0001H     UNIT         ?STACK

            * * * * * * *  X D A T A   M E M O R Y  * * * * * * *
                    0000H     8000H                  *** GAP ***
            XDATA   8000H     000AH     UNIT         ?XD?MAIN

            * * * * * * *   C O D E   M E M O R Y   * * * * * * *
            CODE    0000H     0003H     ABSOLUTE     
            CODE    0003H     004EH     UNIT         ?PR?SPIISR?MAIN
            CODE    0051H     0017H     UNIT         ?PR?CLKCONFIG?MAIN
            CODE    0068H     0001H     UNIT         ?PR?SYSTEMINIT?SYSTEM_FE81001
                    0069H     0002H                  *** GAP ***
            CODE    006BH     0003H     ABSOLUTE     
            CODE    006EH     00F3H     UNIT         ?PR?IOCONFIG?MAIN
            CODE    0161H     009DH     UNIT         ?C_C51STARTUP
            CODE    01FEH     007DH     UNIT         ?PR?MAIN?MAIN
            CODE    027BH     0048H     UNIT         ?PR?SPIMASTERTRANSMITCONFIG?MAIN
            CODE    02C3H     0046H     UNIT         ?PR?_SPI_READBYTE?MAIN
            CODE    0309H     003AH     UNIT         ?PR?_SPI_WRITEBYTE?MAIN
            CODE    0343H     001CH     UNIT         ?PR?DELAY?MAIN
            CODE    035FH     0014H     UNIT         ?C_INITSEG



OVERLAY MAP OF MODULE:   .\Release\Sample_DrvSPI_Master (SYSTEM_FE81001)


SEGMENT
BL51 BANKED LINKER/LOCATER V6.22.2.0                                                  03/13/2023  13:47:56  PAGE 2


  +--> CALLED SEGMENT
---------------------
?C_C51STARTUP
  +--> ?PR?MAIN?MAIN
  +--> ?C_INITSEG

?PR?MAIN?MAIN
  +--> ?PR?CLKCONFIG?MAIN
  +--> ?PR?IOCONFIG?MAIN
  +--> ?PR?SPIMASTERTRANSMITCONFIG?MAIN
  +--> ?PR?DELAY?MAIN
  +--> ?PR?_SPI_WRITEBYTE?MAIN
  +--> ?PR?_SPI_READBYTE?MAIN

?PR?_SPI_WRITEBYTE?MAIN
  +--> ?PR?DELAY?MAIN

?PR?_SPI_READBYTE?MAIN
  +--> ?PR?DELAY?MAIN



SYMBOL TABLE OF MODULE:  .\Release\Sample_DrvSPI_Master (SYSTEM_FE81001)

  VALUE           TYPE          NAME
  ----------------------------------

  -------         MODULE        SYSTEM_FE81001
  C:0000H         SYMBOL        _ICE_DUMMY_
  C:0068H         PUBLIC        SystemInit
  -------         PROC          SYSTEMINIT
  C:0068H         LINE#         38
  C:0068H         LINE#         39
  C:0068H         LINE#         41
  -------         ENDPROC       SYSTEMINIT
  -------         ENDMOD        SYSTEM_FE81001

  -------         MODULE        ?C_STARTUP
  C:0161H         SEGMENT       ?C_C51STARTUP
  I:0012H         SEGMENT       ?STACK
  C:0000H         PUBLIC        ?C_STARTUP
  D:00E0H         SYMBOL        ACC
  D:00F0H         SYMBOL        B
  D:0083H         SYMBOL        DPH
  D:0082H         SYMBOL        DPL
  N:0001H         SYMBOL        IBPSTACK
  N:0100H         SYMBOL        IBPSTACKTOP
  N:0080H         SYMBOL        IDATALEN
  C:0164H         SYMBOL        IDATALOOP
  N:0000H         SYMBOL        PBPSTACK
  N:0100H         SYMBOL        PBPSTACKTOP
  N:0000H         SYMBOL        PDATALEN
  N:0000H         SYMBOL        PDATASTART
  N:0000H         SYMBOL        PPAGE
  N:0000H         SYMBOL        PPAGEENABLE
  D:00A0H         SYMBOL        PPAGE_SFR
  D:0081H         SYMBOL        SP
BL51 BANKED LINKER/LOCATER V6.22.2.0                                                  03/13/2023  13:47:56  PAGE 3


  C:0161H         SYMBOL        STARTUP1
  N:0000H         SYMBOL        XBPSTACK
  N:0000H         SYMBOL        XBPSTACKTOP
  N:0800H         SYMBOL        XDATALEN
  C:016FH         SYMBOL        XDATALOOP
  N:8000H         SYMBOL        XDATASTART
  C:0000H         LINE#         126
  C:0161H         LINE#         133
  C:0163H         LINE#         134
  C:0164H         LINE#         135
  C:0165H         LINE#         136
  C:0167H         LINE#         140
  C:016AH         LINE#         141
  C:016CH         LINE#         145
  C:016EH         LINE#         147
  C:016FH         LINE#         148
  C:0170H         LINE#         149
  C:0171H         LINE#         150
  C:0173H         LINE#         151
  C:0175H         LINE#         170
  C:0178H         LINE#         185
  C:017BH         LINE#         196
  -------         ENDMOD        ?C_STARTUP

  -------         MODULE        MAIN
  C:0000H         SYMBOL        _ICE_DUMMY_
  D:0090H         PUBLIC        P1
  D:00B0H         PUBLIC        P3
  D:00A8H         PUBLIC        IE
  C:027BH         PUBLIC        SPIMasterTransmitConfig
  C:0343H         PUBLIC        delay
  D:00B8H         PUBLIC        IP
  C:01FEH         PUBLIC        main
  D:0098H         PUBLIC        SCON
  C:0051H         PUBLIC        CLKConfig
  D:0088H         PUBLIC        TCON
  D:0008H         PUBLIC        cnt
  X:8000H         SYMBOL        spi_read_data
  X:8005H         SYMBOL        spi_data
  C:0003H         PUBLIC        SPIISR
  C:02C3H         PUBLIC        _SPI_ReadByte
  D:00C8H         PUBLIC        T2CON
  D:0009H         PUBLIC        int_stat
  C:0309H         PUBLIC        _SPI_WriteByte
  C:006EH         PUBLIC        IOConfig
  D:00D0H         PUBLIC        PSW
  D:000AH         PUBLIC        int_stat_1
  D:000BH         PUBLIC        int_stat_2
  -------         PROC          DELAY
  -------         DO            
  D:000CH         SYMBOL        i
  -------         ENDDO         
  C:0343H         LINE#         38
  C:0343H         LINE#         39
  C:0343H         LINE#         42
  C:035EH         LINE#         43
  -------         ENDPROC       DELAY
BL51 BANKED LINKER/LOCATER V6.22.2.0                                                  03/13/2023  13:47:56  PAGE 4


  -------         PROC          SPIISR
  C:0003H         LINE#         55
  C:0012H         LINE#         57
  C:0019H         LINE#         59
  C:0026H         LINE#         61
  C:0033H         LINE#         62
  C:003EH         LINE#         65
  C:0044H         LINE#         66
  -------         ENDPROC       SPIISR
  -------         PROC          SPIMASTERTRANSMITCONFIG
  C:027BH         LINE#         78
  C:027BH         LINE#         79
  C:027BH         LINE#         113
  C:028CH         LINE#         116
  C:0291H         LINE#         117
  C:0297H         LINE#         120
  C:029CH         LINE#         121
  C:02A1H         LINE#         122
  C:02A6H         LINE#         123
  C:02ACH         LINE#         126
  C:02B2H         LINE#         127
  C:02B7H         LINE#         128
  C:02BCH         LINE#         137
  C:02C2H         LINE#         141
  -------         ENDPROC       SPIMASTERTRANSMITCONFIG
  -------         PROC          IOCONFIG
  C:006EH         LINE#         152
  C:006EH         LINE#         153
  C:006EH         LINE#         155
  C:0084H         LINE#         156
  C:009AH         LINE#         157
  C:00B0H         LINE#         158
  C:00C6H         LINE#         161
  C:00E7H         LINE#         162
  C:0108H         LINE#         165
  C:0129H         LINE#         168
  C:014AH         LINE#         171
  C:014FH         LINE#         172
  C:0155H         LINE#         173
  C:015AH         LINE#         175
  C:0160H         LINE#         176
  -------         ENDPROC       IOCONFIG
  -------         PROC          CLKCONFIG
  C:0051H         LINE#         188
  C:0051H         LINE#         189
  C:0051H         LINE#         191
  C:005CH         LINE#         194
  C:0067H         LINE#         196
  -------         ENDPROC       CLKCONFIG
  -------         PROC          _SPI_WRITEBYTE
  D:0010H         SYMBOL        data_
  C:0309H         LINE#         198
  C:030BH         LINE#         199
  C:030BH         LINE#         200
  C:0311H         LINE#         201
  C:0317H         LINE#         202
  C:031DH         LINE#         203
BL51 BANKED LINKER/LOCATER V6.22.2.0                                                  03/13/2023  13:47:56  PAGE 5


  C:0320H         LINE#         204
  C:0331H         LINE#         205
  C:033CH         LINE#         206
  C:0342H         LINE#         207
  -------         ENDPROC       _SPI_WRITEBYTE
  -------         PROC          _SPI_READBYTE
  D:000EH         SYMBOL        dummy
  -------         DO            
  D:000FH         SYMBOL        data_
  -------         ENDDO         
  C:02C3H         LINE#         209
  C:02C5H         LINE#         210
  C:02C5H         LINE#         211
  C:02C8H         LINE#         212
  C:02CEH         LINE#         213
  C:02D4H         LINE#         214
  C:02DAH         LINE#         215
  C:02DDH         LINE#         216
  C:02EEH         LINE#         217
  C:02F9H         LINE#         218
  C:0300H         LINE#         219
  C:0306H         LINE#         221
  C:0308H         LINE#         222
  -------         ENDPROC       _SPI_READBYTE
  -------         PROC          MAIN
  C:01FEH         LINE#         235
  C:01FEH         LINE#         236
  C:01FEH         LINE#         237
  C:0201H         LINE#         238
  C:0204H         LINE#         240
  C:0207H         LINE#         242
  C:020AH         LINE#         244
  C:020AH         LINE#         245
  C:020AH         LINE#         246
  C:0221H         LINE#         247
  C:0221H         LINE#         248
  C:0238H         LINE#         250
  C:023DH         LINE#         254
  C:0242H         LINE#         256
  C:0247H         LINE#         257
  C:024CH         LINE#         258
  C:0251H         LINE#         259
  C:0256H         LINE#         261
  C:0260H         LINE#         262
  C:026AH         LINE#         264
  C:0270H         LINE#         266
  C:0272H         LINE#         268
  C:0272H         LINE#         269
  C:0278H         LINE#         270
  C:0278H         LINE#         271
  -------         ENDPROC       MAIN
  -------         ENDMOD        MAIN

  -------         MODULE        ?C_IBP
  D:0011H         PUBLIC        ?C_IBP
  -------         ENDMOD        ?C_IBP

BL51 BANKED LINKER/LOCATER V6.22.2.0                                                  03/13/2023  13:47:56  PAGE 6




FUNCTION REGISTER MASKS


FUNCTION . . . . . . . . . REG MASK
-----------------------------------

CLKCONFIG. . . . . . . . . @0xe301
DELAY. . . . . . . . . . . @0xf000
IOCONFIG . . . . . . . . . @0xe301
MAIN . . . . . . . . . . . @0xf303
SPIISR . . . . . . . . . . @0xe303
SPIMASTERTRANSMITCONFIG. . @0xe303
SYSTEMINIT . . . . . . . . @0x8000
_SPI_READBYTE. . . . . . . @0xf303
_SPI_WRITEBYTE . . . . . . @0xf303

*** WARNING L16: UNCALLED SEGMENT, IGNORED FOR OVERLAY PROCESS
    SEGMENT: ?PR?SYSTEMINIT?SYSTEM_FE81001

Program Size: data=19.0 xdata=10 code=881
LINK/LOCATE RUN COMPLETE.  1 WARNING(S),  0 ERROR(S)
